:020000040000FA
:1000000008030020F9000000FD000000DD000000F2
:1000100000000000000000000000000000000000E0
:1000200000000000000000000000000001010000CE
:1000300000000000000000000301000005010000B6
:100040000701000007010000810A00009D0A00006E
:100050000701000007010000070100000701000080
:10006000F50E0000110F000007010000070100005D
:100070002D0F00000701000007010000070100002C
:100080000701000007010000070100000701000050
:100090000701000007010000070100000701000040
:1000A0000701000007010000070100000701000030
:1000B0000701000007010000070100000701000020
:1000C0000348854600F040FA00480047C91F000079
:1000D00008030020401EFDD2704700000420714636
:1000E000084202D0EFF3098001E0EFF30880714687
:1000F000004A1047710B000003480047FEE7FEE787
:10010000FEE7FEE7FEE7FEE7C100000030B50B4664
:10011000014600202022012409E00D46D5409D42E1
:1001200005D31D469540491B254695404019154667
:10013000521E002DF1DC30BD03460B439B0703D05C
:1001400009E008C9121F08C0042AFAD203E00B789C
:100150000370401C491C521EF9D27047F0B51FB401
:100160000646002082B005464024019100901BE025
:10017000019922460F46304600F008FA049A059B82
:10018000801A994110D310461946224600F0EEF924
:10019000361A8F410197224601200021009F00F06E
:1001A000E5F938184D4100902046641E0028DFDC38
:1001B000019B00982946324607B0F0BDF0B50746CE
:1001C0000846584087B0C00F049048000E465900BA
:1001D00040084908BC1A884105D2384631461E46B7
:1001E00017460B4602465800400810434CD0300DCD
:1001F000039040055900400D490D0590401A0290AA
:10020000402872DA18030121000B09050843019008
:1002100004980092002805D001995242002088419C
:1002200000920190029840210A1A0199009800F06A
:100230009DF905460C466B4607CB00F0B8F9C0198E
:100240007141039A0E0D0023D71756401A467A4083
:10025000164344D0049A002A2DD0029A012A039A08
:1002600015DC1205C01A914101263605001C7141AA
:10027000D20F059ED2070093019202962A4623468A
:1002800000F0B5F907B0F0BD38463146FAE716057B
:10029000224A0F46B218C01AB74101210905001CB5
:1002A0004F4100187F41114618187941E20F104361
:1002B0006D19644113E0E2076D0815436408C20735
:1002C0001443039A01261205C01A91413605001CF9
:1002D0007141CE07400830434908C01851412A46B1
:1002E000234600F077F9CDE7FFE7049801224000AC
:1002F000C117121A00238B4104983146C417381ACB
:10030000A141EEE730B40124E407634030BC55E777
:1003100030B40124E407614030BC4FE70000E0FF47
:10032000F0B51FB488B00B9909980024484009998A
:10033000C00F490049080991C0070B990090490076
:1003400049080B9109990898A64608431CD00B99B7
:100350000A98084318D0099801244000420D48002B
:10036000410D099824050003000B204309900B98C8
:100370000003000B20430B9050181C49401800222A
:1003800001901446104605E0002001460DB0F0BD76
:10039000032801DA034600E003239C46C11A0AAE93
:1003A0000AE05F0008ADED5B4F00F75B7D4300277F
:1003B000AA187C41491C5B1E6145F2DD410004AB7B
:1003C0005A522104120C0A43240C401C0828DFDB7B
:1003D000019802900099704601910090059B049A43
:1003E0000799069800F003F9D0E700000DFCFFFF25
:1003F000F0B50C465C4085B0E40FE40703944C0074
:100400000026640859009446490802460296224391
:1004100021D062460A431ED06200570D4A000E03E7
:100420002303550D012402462C492405781B1B0B80
:10043000360B401823432643614600901C46501A51
:10044000B44103D30098401C009002E09218009839
:100450005B41002803DA0020014605B0F0BD002012
:10046000012109050746864611E064461D46141B16
:10047000B54106D36546521BB341744607430C434E
:10048000A646CD0740084908284392185B41054617
:100490000D43EAD11046184313D060461946504028
:1004A0007140084306D06046101AB34106D20122BB
:1004B000002306E000220123DB0702E00122D243F1
:1004C0005310009874460105381C6141029C039D3D
:1004D0000019694100F07EF8BFE70000FD0300004D
:1004E0004A0009030123090B1B0519430A4B10B5E8
:1004F000520D9A4202DA0020014610BD064B3433F9
:100500009A4203DC9A1A00F041F810BD034BD2184E
:1005100000F02CF810BD0000FF030000CDFBFFFF32
:1005200010B5002904DB0124E40740428C41214638
:10053000002B04DB1C460123DB075242A3419942F6
:1005400000D1904210BD0000064C0125064E05E08A
:10055000E36807CC2B430C3C98471034B442F7D3E4
:10056000FFF7B2FD142900003429000010B5202A3D
:1005700004DB0146203A9140002010BD9140202329
:100580009C1A0346E3401943904010BD10B5202A41
:1005900004DB0846203AD040002110BD0B46D34072
:1005A000D0402024A21A91400843194610BD10B52E
:1005B000202A06DBCB170846203A1041C1170B430F
:1005C00006E00B461341D0402024A21A9140084374
:1005D000194610BD10B5002B08DA0024401C6141FB
:1005E00092185B411A4301D14008400010BDF0B59C
:1005F0001FB482B005460C0003D0084600F02EFD63
:1006000002E000F02BFD20300246009021462846F3
:10061000FFF7ACFF049B059A04460F4618431143AD
:10062000084314D0184610431BD0009840210A1AE2
:1006300018460599FFF7AAFF05460E46009A059948
:100640000498FFF793FF084305D0012004E02046FB
:10065000394607B0F0BD0020C11705430E432C43B7
:10066000374300990E986305401A7905E40A002281
:100670000C43FD0A0A3002D500200146E9E70105D6
:10068000101969410C9C0D9D00196941FFF7A2FFEB
:10069000DFE700000248016AC201114301627047AE
:1006A00000020050C10F8A00044951184A68C3066D
:1006B000DB0E0120984002434A6070470002005060
:1006C000F3B58BB00C46FFF7E5FF0B980028744894
:1006D000016813D0042211430160102000F0BCF91E
:1006E0000120C00409906F480090042008906E48D3
:1006F0006E49201888420ED800251DE0890889001F
:10070000491C0160012000F0A7F900200990684809
:1007100000900220EAE7674866492018494288426B
:1007200002D80125640007E0634863492018494264
:1007300088427DD20325A4000026F643089F22E0CC
:1007400039460098FFF7E2FC5C49844641185C4852
:10075000814217D2554B02225B1C534861465143DC
:10076000401C0818984209D8A14201D9081B00E092
:10077000601AB04202D2060004920CD05148521CBA
:100780008242EAD97F1C212FDAD900200696C04385
:100790000190089E54E00999A803084301217A02B8
:1007A0008902511A08430499891E08433C4908628A
:1007B000042000F051F9691C79430098FFF7A6FC6A
:1007C000049948430DB0F0BD31460098FFF79EFCF8
:1007D0003A4942183A498A4231D20221324B024602
:1007E0004A435B1CD7185B429F4224D8A24201D9DE
:1007F000121B00E0A21A019B9A421CD20192069B96
:100800000F469A4217D10999A803084301217202A1
:100810008902511A0843B91E08432149086204207D
:1008200000F01AF9691C71430098FFF76FFC00E0B3
:1008300008E07843C6E7234A491C9142CED9761C8A
:10084000212EC1D90B9800280FD01F4914480162EE
:10085000042000F001F91DA0006803901048016A0F
:100860000013014203D00020ACE71949EEE708036A
:1008700001D50C4800E00E488A03A3D40A04920F65
:1008800003AB9B5CCA058904D20DC90E891C800884
:10089000921C59435043FFF739FC800092E7000057
:1008A0000002005000805101FF1E0AFAFFE0F5052A
:1008B000001BB700800F05FDC08782FEFF95E7FF94
:1008C000BF77CC00010200001844080001020204B6
:1008D00016400000044982070A6801D0920892007D
:1008E00002430A60704700000002005010B500F09B
:1008F0005DFA0148006810BD080000200448006847
:100900008007800F012801D0002070470148704700
:1009100000020050001BB700044800688007800FE9
:10092000022801D0002070470148704700020050A3
:10093000001BB70008B511A0006800901048016ABC
:100940000013014201D0002008BD080301D50D4865
:1009500000E00D488A03F7D40A04920F6B469B5CB3
:10096000CA058904D20DC90E891C8008921C5943FE
:100970005043FFF7CBFB800008BD000001020204DA
:100980000002005000805101001BB70008B511A003
:10099000006800901048016A0013014201D0002055
:1009A00008BD080301D50D4800E00D488A03F7D4BF
:1009B0000A04920F6B469B5CCA058904D20DC90ECE
:1009C000891C8008921C59435043FFF79FFB80000D
:1009D00008BD000001020204000200500080510125
:1009E000001BB70010B5074A93691B091B010B4395
:1009F00093611169C908C9000143116100F0D6F97A
:100A000010BD00000002005070B5430E1B070DD052
:100A100043009B0F0F4C9B001C192368C5002D0F32
:100A2000C601F60EB540AB430B432360840A210692
:100A3000090E0DD00103074B890F89000833CB182D
:100A400019688005E4B2C00E8440A14311431960C7
:100A500070BD00001002005010B50749074A05E0BC
:100A60000B46491E002B01DC002010BDD468034654
:100A7000A343F5D1012010BD80F5200000020050F5
:100A800004490420086204484068002800D0004758
:100A900070470000C040005054000020044904206A
:100AA000086204480068002800D000477047000032
:100AB00040410050540000200248016849084900A4
:100AC0000160704700C000500A492222CA60486095
:100AD000012008610869C007FCD10868400606D5F6
:100AE00008684022104308600020C043704700207F
:100AF0007047000000C00050024801680122114305
:100B00000160704700C0005005490022CA6048607B
:100B1000012008610869C007FCD18868704700009F
:100B200000C00050054A2123D3605060916001202D
:100B300010611069C007FCD17047000000C0005070
:100B4000F0B500230125944603272A469A400A421D
:100B500009D006685C003A46A240964322466446A5
:100B60009440264306605B1C082BEED3F0BD0000CA
:100B7000044603A000F052FA204601F059FCFEE7BB
:100B8000496E2048617264204661756C742048612A
:100B90006E646C65720A00008307FF22DB0E9A40C8
:100BA0008907090E994000280BDA0007000F083862
:100BB000830808489B001818C36993430B43C3611B
:100BC0007047830804489B001B181868904308432B
:100BD0001860704700ED00E000E400E08168082242
:100BE00091438160704710B5029C202B00D10023F7
:100BF000DB000B431343036001229204914201D1B5
:100C000010218160214600F001F810BD70B5064644
:100C100019480D4641698906890F21D0406980062F
:100C2000800F022823D0FFF761FE0446A54200D9B9
:100C30000546002D1ED029462046FFF767FA401CC6
:100C40004008401EFF2800D9FF207168090A0902E8
:100C50000143716041002046891CFFF757FA70BDBF
:100C6000FFF74CFE0400E1D1FFF756FEDDE7FFF78A
:100C70008DFEDAE7002070BD00020050F8B5592162
:100C8000304C162288202160226020602368002BCF
:100C9000F9D02D4D04202860FFF71CFE0820FFF737
:100CA00019FE1020FFF7D8FE2869072108432861A4
:100CB000A86900090001A8612449A802FFF700FD06
:100CC00001210220FFF78EFE2148FFF7EBFC214EA9
:100CD0003046FFF7E7FCB322120408213046FFF745
:100CE00093FE1D48FFF7DEFC1C48FFF7DBFC00F01D
:100CF0005DF81BA000680090286A291301400025B8
:100D0000002901D02A4616E0010301D5154A00E06A
:100D1000154A81030FD40104890F6B465E5CC3053D
:100D20008004C10EDB0D891C90089B1C7143584345
:100D3000FFF7ECF982000D4EB260FFF7D7FDF060CF
:100D40002560F8BD000100500002005000E1F505EB
:100D5000103D80A71CFE23A61400C0A71500E0A725
:100D60000102020400805101001BB70010000020A6
:100D700010B55921044816228823016002600360DF
:100D80000468002CF9D010BD0001005006498A69A2
:100D90001202FCD408600A2804D188690002FCD43D
:100DA0000D2008607047000000000540F8B520A045
:100DB0000068204E0090316A30131F4C1F4F0142D3
:100DC00001D0002016E0080301D5204600E0384697
:100DD0008A030FD40A04920F6B469B5CCA058904F0
:100DE000D20DC90E891C8008921C59435043FFF74D
:100DF0008DF98000124D286031694907490F12D0E2
:100E0000022902D0032910D02046B1690907090F31
:100E1000491CFFF77BF90B4968604A108018FFF7FF
:100E200075F9A860F8BD3846EFE70748EDE7000020
:100E3000010202040002005000805101001BB700B3
:100E40000400002040420F00102700000F4A104904
:100E50009042486901D1000A00E0000B4007400FB2
:100E600006D001280ED002280ED00A48006870472C
:100E700008688007800F012802D00120C003704756
:100E800005487047054870470548EFE700000140F6
:100E90000002005000000020001BB70010270000D7
:100EA00008000020F8B513460F460646FFF7CEFFB0
:100EB000044600254008984201D2022010E001219A
:100EC00049068C4202D30325A40805E00121090646
:100ED0008C4201D30125044619462046FFF716F936
:100EE0002F43376070606D1C684301462046FFF752
:100EF0000DF9F8BD04490120886004480068002805
:100F000000D0004770470000000001405C00002056
:100F100004490120886004484068002800D0004748
:100F200070470000200001405C00002070B51849A7
:100F3000CD690022EB05174C1748002B0BDB0DE0A9
:100F40000378202B04D20E68E6545B1C037002E089
:100F500002700B682370CB69DB07F1D1AB0515D5A7
:100F600043888488A34211D2002C0FD0094D20352C
:100F7000ED5C5B1C45709BB243800D60A34205D3C2
:100F800082804280486802229043486070BD000021
:100F900000000540B00000206400002070B51B4E2A
:100FA0000D4604467169002089010322890F2063E0
:100FB000E260A06000291FD001291FD0022901D3BF
:100FC00013480068B1690905090F491CFFF79EF82D
:100FD0000646002D19D0680880192946FFF796F8B3
:100FE0000C49801E88420CD9E80080192946FFF779
:100FF0008DF80009801E07E00748E3E7FFF79AFC39
:10100000E0E7032109070843606270BD0002005059
:1010100000000020FFFF0000001BB7000FB410B558
:1010200003A9044B044A029800F0E4FA10BC08BC7F
:1010300004B018472D1F00006C0000200FB410B53D
:1010400003A9044B044A029800F066F910BC08BCDE
:1010500004B018472D1F00006C0000202021020C56
:1010600001D010211046020A01D0104608390209A9
:1010700001D01046091F820801D01046891E42087F
:1010800001D0881E7047081A704702E008C8121F76
:1010900008C1002AFAD170477047002001E001C161
:1010A000121F002AFBD1704710B504460089FFF7D4
:1010B00011F86168012008606089FFF70BF861682A
:1010C000002008602089FFF705F810BD70B50446C0
:1010D0000068012505602089FEF7FCFF6068056057
:1010E0002089FEF7F7FF206800686168C5B200201C
:1010F00008602089FEF7EEFF284670BDF8B500268F
:1011000004463546374676002089FEF7E3FF6168DE
:10111000012008602089FEF7DDFF20680068304369
:10112000C6B2606807602089FEF7D4FF6D1CEDB27F
:10113000082DE8D33046F8BD70B50446216801207B
:101140000860616808602089FEF7C4FF20680025F8
:1011500005602089FEF7BEFF606805602089FEF704
:10116000B9FF70BD70B50446216800200860606852
:10117000012505602089FEF7ADFF2068056070BD80
:1011800070B506460D4600243168E809086030460F
:10119000FFF78AFF6806641C050EE4B2082CF3D33F
:1011A00070BD0000F0B51FB486B00998089A030D11
:1011B0000021024314D05148514A181850430514D5
:1011C0001198012810981AD0281A401C00264D4F5B
:1011D0004D49009601910490002812DA444211E032
:1011E0001198012449A3012801D11098C143069800
:1011F000119A84600360C26041600BB0F0BD404250
:10120000E4E70446210500203F4A001C51410391B8
:10121000029012E0E00707D032463B460199009861
:10122000FFF77EF80191009032463B461046194682
:10123000FFF776F806460F466410002CEAD10498B2
:10124000039B0028029A0999089806DAFFF768F8C4
:10125000019B009AFFF764F805E0FFF7C9F8019BCE
:10126000009AFFF7C5F804460E460022284BFFF708
:1012700057F903D80020C043014607E00022254B60
:1012800020463146FEF79AFFFFF72AF9102409E0BD
:10129000002C0ADB0A220023FEF760FF079B303296
:1012A0001A55641E02460A43F2D11122641C079BA0
:1012B000121B1C19119B012B03D0012308430ED1D3
:1012C0000AE0084304D0112010900020119077E725
:1012D0001098151A6D1E0BE01098824202DD002353
:1012E0006D1C03E0824201DA00236D1E002BEED05C
:1012F000069811998260C16030C07EE701FCFFFF53
:10130000104D0000000014400000F03F30000000CD
:101310000000F0430000E03FFFB58FB00F460446E9
:10132000002606E025280AD0129A11999047641CDD
:10133000761C20780028F5D1304613B0F0BD00258A
:101340000121A14A009500E00543641C237808466A
:10135000203B98401042F7D120782E2815D1042048
:1013600005436078641C2A280AD101CF641C0090D0
:101370000BE000990A22514330394018641C009058
:101380002078014630390929F3D920786C280ED00D
:1013900004DC4C2813D06A2812D104E074280ED043
:1013A0007A280DD10BE001204005054307E001211B
:1013B000090562780D43824201D16D18641C641CDA
:1013C0002078864669284AD008DC0028B4D05828FE
:1013D0006DD0632810D0642808D140E070286BD00D
:1013E000732812D0752860D0782860D0129A704681
:1013F00011999047761CE5E038786946087200201C
:10140000487202A80190012003E038680190002092
:10141000C0433F1D69070CD5002500E06D1C0099F5
:101420008D420FDA8542F9DB0199495D0029F5D13A
:1014300008E0002500E06D1C8542FCDB0199495D58
:101440000029F8D1761907E0019801990078491C24
:101450000191129A119990476D1EF5D2B2E00A20BF
:10146000029000216802400F039102280CD001CFA6
:10147000C117844600290DDA62460846524200210F
:10148000814194462D2008E0FF1DFF08FF0003CF97
:101490008446EFE7280504D52B206A461074012006
:1014A0003CE0E8073AD02020F7E70A2000E01020CF
:1014B00000210391029007E01020029000210420F7
:1014C00005430820039100906802400F022810D0C5
:1014D00001CF0021844600200D9028071FD57046BB
:1014E00070280CD0029A1020039B42401A430CD063
:1014F00015E0FF1DFF08FF0003CF8446EBE7402007
:101500006A46107401200D900CE06046084306D036
:1015100030206A4610747046507402200D90704658
:10152000582804D029A001900DA80E900DE02CA001
:10153000F9E76046039B029AFEF710FE019B844682
:101540009B5C0E9A521E0E92137060460843F0D1B7
:101550000E9805A9081A20300190680701D5009857
:1015600001E0012000900199884203DD01460198C5
:10157000081A00E000200025009006E004A8129A56
:10158000405D119990476D1C761C0D988542F5DBE6
:1015900004E0129A302011999047761C0099481E59
:1015A00000900029F5DC08E00E980E990078491C9F
:1015B0000E91129A11999047761C0199481E01903C
:1015C0000029F1DC641CB4E6092801003031323313
:1015D000343536373839616263646566000000006F
:1015E0003031323334353637383941424344454659
:1015F00000000000FFB597B00646002518E2252838
:1016000077D100242746FD49049400E00443761C6A
:1016100032780120203A90400842F7D130782A28C9
:101620000ED00222307801463039092916D80499A3
:101630000A235943303940181443761C0490F1E7CB
:10164000189802C804911890002904DA0120400378
:1016500004434842049002200443761C30782E282C
:1016600014D1042004437078761C2A2809D11898D4
:10167000761C80C8189009E00A214F43303FC719F3
:10168000761C3078014630390929F5D930786C2834
:1016900010D006DC4C281AD068280ED06A2817D142
:1016A00004E0742813D07A2812D110E001204005FC
:1016B00004430CE00121090501E0032109050C4365
:1016C0007178814203D1012000052418761C761C14
:1016D0003078119066280BD013DC58287DD009DCB7
:1016E00000287BD04528F6D04628F4D047281AD1C8
:1016F000A5E118E0632835D0642870D0652812D1A0
:101700009DE170286CD008DC6728F1D069287BD077
:101710006E280DD06F2806D1BAE073282ED0752818
:1017200071D0782859D01A9A199990476D1C7EE18A
:101730006002400F022809D003280DD00428189811
:1017400001680DD00D60001D189070E11898EA171F
:1017500001680D604A60F6E7189801680D80F2E7AD
:101760000D70F0E718986A4601781172001D189004
:101770000020507202A80090012005E0189802C8CD
:10178000189000200091C04361070DD5002101E0B1
:101790000199491C0191B94212DA8142F8DB009AA1
:1017A000515C0029F4D10BE0002101E00199491CB2
:1017B00001918142FADB019A0099895C0029F5D1F7
:1017C000019904981A9B471A21463846199A00F045
:1017D00097FA0199401945180BE04FE02CE113E00E
:1017E0004EE0009800990078491C00911A9A1999C6
:1017F00090470198401E0190401CF2D12146384686
:101800001A9B199A10E137E00A20002100900191FB
:101810006002410F022907D0189A01CA1892C21714
:101820009446032908D00AE01898C01DC108C900D1
:1018300005C91891944607E000B2C21794460429DE
:1018400002D140B2C1178C4600226146944506DAA7
:101850000A460021404291418C462D2102E021059B
:1018600004D52B216A461173012103E0E10701D061
:101870002021F7E7029155E00A200AE0102008E055
:10188000102000900021042004430191082703E068
:1018900008200021019100906002410F022907D029
:1018A000189A01CA189200229446032908D008E029
:1018B0001898C01DC108C90005C91891944603E0D5
:1018C00080B2042900D1C0B200210291210729D59C
:1018D0001199702906D0009A1021019B4A401A43A1
:1018E00005D00EE040216A461173012108E06146EF
:1018F000014306D030216A461173119951730221B8
:101900000291009A0821019B4A401A430AD161467C
:10191000014301D1610705D530216A4611730121C8
:101920007F1E02911199582904D035A10E910DA95D
:101930000D910DE037A1F9E76146019B009AFEF792
:101940000DFC0E9B8C469B5C0D9A521E0D921370E3
:1019500061460143F0D10D9805A9081A2030019085
:10196000600703D501200004844300E001270198AB
:10197000874201DD381A00E00020019900904118EB
:10198000029809180498401A0490E00306D42146EE
:101990001A9B199A049800F0B3F94519002706E03C
:1019A00003A81A9AC05D199990476D1C7F1C029874
:1019B0008742F5DBE0030CD521461A9B199A04985F
:1019C00000F09EF9451904E01A9A302019999047C1
:1019D0006D1C0099481E00900029F5DC08E00D9868
:1019E0000D990078491C0D911A9A199990476D1C10
:1019F0000199481E01900029F1DC63E109280100EA
:101A00003031323334353637383961626364656674
:101A10000000000030313233343536373839414236
:101A2000434445460000000000F05AF94519761C71
:101A30003078002800D0E2E528461BB0F0BD6007F2
:101A400000D406271898C01DC108C90048680A6854
:101A50000831C30FDB071891190001D09CA108E0E1
:101A6000210501D59BA104E0E10701D09AA100E086
:101A70009AA1430011985B08109165280CD006DCF0
:101A8000452809D046281DD0472841D141E0662885
:101A900018D067283CD13CE00021112F01DB112038
:101AA00000E0781C0191009008A911A8FFF77AFBCB
:101AB000139905910021119A15927F1C1298019794
:101AC000009150E00120C00703900120019008A977
:101AD000009711A8FFF766FB139A1499059200224C
:101AE000119B009212981593059A0192002901D03A
:101AF000104602E0791C40180190381A01D501986F
:101B000004E04042401E0090781C0190C01B0290EF
:101B100043E0012F00DA01270021112F01DD112000
:101B200000E038460191009008A911A8FFF73AFBA0
:101B300013990591119A002112981592009101971D
:101B400021070CD40599B94201DB019900E001910C
:101B5000012904DD159A491E515C302906D0B8428E
:101B600001DA011D05DA0121029115E00199491EF2
:101B7000EDE7002805DC0099411800910199091A48
:101B800003E0019A411C914200DD01910099401A45
:101B9000401C02900120C0070390200706D4029940
:101BA0000198814202DB0020C04302900020694678
:101BB000C87707AF012103980337C907884224D0AB
:101BC000022011902B201290039800280CDA40423A
:101BD00003902D20129007E00A210398FEF796FA51
:101BE00030317F1E039039701199481E11900029E1
:101BF000F2DC03980028EFD1791E12980870307833
:101C0000202108404530BF1E387006A8C01BC01DEB
:101C1000039010980078002800D001200199411805
:101C20000298C0170918039809180498401A401E12
:101C30000490E00306D421461A9B199A049800F0F8
:101C40005FF8451910980078002803D01A9A19995E
:101C500090476D1CE00324D521461A9B199A0498DD
:101C600000F04EF845191CE00098002807DB0099A9
:101C70000598884203DD1598405C199901E019998F
:101C800030201A9A904700986D1C401C00900298D2
:101C9000401E0290002804D11A9A2E2019999047CC
:101CA0006D1C0199481E01900029DDDC05E03878A3
:101CB0001A9A7F1C199990476D1C0399481E03902E
:101CC0000029F4DC21461A9B199A0498ACE600001E
:101CD0002D0000002B00000020000000000000008C
:101CE000F8B5044600251E461746880404D405E0CE
:101CF00039462020B0476D1C641EF9D52846F8BD32
:101D0000FFB50446002581B01E46C80301D5302723
:101D100000E02027880404D505E038460399B04741
:101D20006D1C641EF9D5284605B0F0BD0A48016A4D
:101D300001221143016205200007416B074A11404F
:101D40004163416B08221143416305484168120415
:101D5000114341607047000000000E40F7F7FFF7A5
:101D6000404000500B4908224A620A4A40329368B8
:101D70001B091B019B1D93600A6A0123DB021A43A6
:101D80000A620A6B1207FCD409688905890D018073
:101D90007047000000000E4010B505200007816B61
:101DA0008163C16BC163012240210748FEF7C8FE71
:101DB0000548012202214030FEF7C2FE03480021FF
:101DC0008161416210BD00008040005040420050DF
:101DD000F8B50D460646FEF7CBFFFEF78DFE0B4C21
:101DE000206804273843206005E03046FEF76CFE8B
:101DF0006D1EADB28036002DF7D12068B84320604B
:101E0000FEF75AFE024900200860F8BD00C00050ED
:101E100000010050F7B582B015460E46FEF7A8FF48
:101E2000FEF76AFE1C480168042211430160002489
:101E3000AF0809E00298FEF767FEA1007050029813
:101E4000001D641CA4B20290A742F3D8A004040CA5
:101E5000AC4214D20298FEF757FE00906846007814
:101E60003055641CA0B2A84209D269464978315461
:101E7000401C80B2A84202D2694689783154064893
:101E80000168042291430160FEF716FE0349002019
:101E9000086005B0F0BD000000C000500001005017
:101EA000F7B5002082B0C04315460E460090FEF7FD
:101EB0005FFFFEF721FE1B48016804221143016009
:101EC0000024AF0809E0A00031580298FEF72AFE6E
:101ED0000298001D641CA4B20290A742F3D8A0048B
:101EE000000CA84212D2315C401C6A4680B21170CC
:101EF000A84207D2315C401C80B25170A84201D286
:101F0000305C907000990298FEF70CFE054802685C
:101F100004218A430260FEF7CFFD034900200860D8
:101F200005B0F0BD00C000500001005000B50346F0
:101F3000FEF72CFF184600BD1CB503200521084CF8
:101F400002460191009004232146064800F0CCFA95
:101F50000449224608460C3000F0BEFA1CBD0000C1
:101F600003000300F0000020F8B50E460093C1B254
:101F70001346069D079C3246064800F0E5FA002805
:101F800003D0002D00D0A847F8BD002CFCD0A047FE
:101F9000F8BD0000F0000020F8B50E460093C1B275
:101FA0001346069D079C3246064800F01AFB00289F
:101FB00003D0002D00D0A847F8BD002CFCD0A047CE
:101FC000F8BD0000F00000201FB5FEF757FEFFF738
:101FD000B3FF00F0C7F9012000F0B4F8FFF7A6FE48
:101FE00000F0ACF900F058FBFF204B49F53000F051
:101FF00029FB4AA0FFF722F800F08EF9FFF7CCFE8C
:1020000001214C052046FFF7E3FE0D2247492046FB
:10201000FFF746FF0D2245492046FFF7FBFE00F083
:1020200045FC3127424D002440480321183800F078
:102030005BFB0D213D4800F017FC3C480C38FFF7D6
:1020400091FE3A4E1C3E3078401CC0B230700128E0
:1020500004D0022807D0032814D10CE03348C8214B
:102060000838418002E03148083844802F48083859
:1020700000F020F907E02D48192149010838418076
:1020800000F018F934702BA103C9009402AA01943E
:1020900003C201230C217620083AFFF77DFF3E465C
:1020A0002846FEF717F8761EFAD200941223234A28
:1020B000102176200194FFF757FF00262846FEF7EF
:1020C00009F8761EFAD2009412231C4A10217620B9
:1020D0000194FFF749FF00262846FDF7FBFF761E17
:1020E000FAD200941223154A102176200194FFF7AA
:1020F0003BFF00262846FDF7EDFF761EFAD210487A
:102100000090019030230D4A10217620FFF72CFF1C
:1021100072B662B688E700000D2400006164632097
:1021200076616C7565206973000000002C0000204A
:10213000086100008902030405000000700000200F
:1021400001240000F8B504465920524D162288217A
:1021500028602A6029602B68002BF9D04E48FEF7D2
:10216000A1FA4E48FEF79EFAFEF720FE00232B60F0
:1021700005221207906B4A4908409063916B012039
:1021800080020143916347498D68092635438D607C
:10219000956B454E35409563956B46003543956389
:1021A0008D68902635438D60956B404E3540956324
:1021B000956B8600354395638D6809263602354355
:1021C0008D60956B3A4E35409563956BC6003543EF
:1021D00095638A6809252D032A438A600D68FF22CA
:1021E00012029543260235430D604D6807273F02D2
:1021F000BD43281848608868400040088860CB626A
:102200007D20C00048610D682D0A2D0225430D6018
:102210004D687027BD4340354D608D686D006D0879
:102220008D608B6208610D682D0A2D0225430D60BB
:102230004C68E408E400241D4C608C686400640869
:102240008C604B62C8600C68944334430C604A68ED
:102250003C02A2430124A40312194A608A68520076
:1022600052088A600B638861886801221043886085
:10227000886810221043886088688A151043886037
:1022800088681201104388604B628B62CB620B63DB
:10229000F8BD0000000100501400C0A71500E0A721
:1022A000FBFBFFFF00000440F7F7FFFFEFEFFFFF2E
:1022B000DFDFFFFF30B5174B0022048811469C6218
:1022C0000488002C1ED0022144881C634588082401
:1022D000002D19D021438488DC6285880424002DD8
:1022E00014D02143C4885C62C3880120002B0FD026
:1022F000014308484030C3699343C361C2690A433C
:10230000C26130BD0222DFE72243E4E72243E9E76E
:102310000243EEE7000004401CB507A000680190EE
:102320006720009020230222032101A800F002FA76
:1023300000F0BCFA1CBD0000A55A11001CB508A095
:102340000068019000F00EF82C2000900D2314225C
:10235000032101A800F0EEF900F07CFA1CBD00009A
:1023600023232300F8B505242407206B2063206B6A
:1023700007256D0328432063134841684160134ECD
:102380003046FEF78FF9012210213046FEF73CFB64
:10239000012202210E48FEF7D3FB002204210D4842
:1023A000FEF7CEFB206B284320630B480B4C0090BC
:1023B0000823042200212046FEF715FC2046FEF7E4
:1023C0000DFC00202062F8BD400000500C0040A62B
:1023D000004000504041005080841E000000034037
:1023E0000649086208680122104308600868C04373
:1023F000C007FBD00869C0B270470000000003406E
:102400000149012048807047100000201CB5064992
:10241000022048800020009001901223034A1021DE
:102420007620FFF7A1FD1CBD1000002070000020E9
:1024300010B50446016810A0FEF7F0FD11A0616818
:10244000FEF7ECFD12A0A168FEF7E8FD13A0E1681D
:10245000FEF7E4FD14A02169FEF7E0FD15A0616917
:10246000FEF7DCFD16A0A169FEF7D8FD17A0E16913
:10247000FEF7D4FD10BD0000723020203D203078E2
:1024800025780A00723120203D20307825780A0016
:10249000723220203D20307825780A0072332020C7
:1024A0003D20307825780A00723132203D20307886
:1024B00025780A006C7220203D20307825780A00AB
:1024C000706320203D20307825780A0070737220D8
:1024D0003D20307825780A0010B51AC91AC00C388A
:1024E000511C00D0826010BDF8B58C4605465001E5
:1024F000990041181348069F0918079E29607C011E
:10250000B1006118081868600124604621469940AE
:10251000A8609001A203104305221207801802222E
:10252000FEF70EFBB4400122B801920310430522CE
:102530001207801821460222FEF702FB2846FEF70A
:1025400011FEF8BD00420050FFB581B01F460E4697
:102550000546002472B6FEF7EFFD7600F1B228467C
:10256000FEF70EFE2846FEF7B1FD002832D12846C0
:102570000399FEF705FE2846FEF7A8FD002829D19D
:102580002846FEF7D9FD761CF1B22846FEF7F8FD85
:102590002846FEF79BFD00281CD10A9E761E0CE003
:1025A000FEF7ACFD38552968002008602846FEF784
:1025B0007BFD296801200860641CB4422846EFD3E3
:1025C000FEF79CFD38552968012008602846641CE8
:1025D000FEF76AFD2846FEF7C5FD62B6204605B047
:1025E000F0BDFFB581B00A9F1D460E46002472B6AD
:1025F0000198FEF7A1FD7006010E0198FEF7C0FDDF
:102600000198FEF763FD002815D103990198FEF7A4
:10261000B7FD0198FEF75AFD00280AD00BE0295DAE
:102620000198FEF7ADFD0198FEF750FD002802D19C
:10263000641CBC42F3D30198FEF794FD62B62046B9
:1026400005B0F0BD70B504460D460F48FEF72AF8F8
:1026500022460E4C0121C9062046FEF723FC002D20
:102660000AD02068610308432060481508490860C3
:1026700002210820FEF790FA064805602068012133
:1026800089070843206070BD020080AE0000014051
:1026900000E100E05C00002010B50D48FEF702F8F4
:1026A0000D490C4848600D4841680122520491438D
:1026B00041600B4CE12149022046FEF76FFC606847
:1026C000112108436060012006490003086010BD25
:1026D000103D80A70303000040000050404100501F
:1026E0000000054000E100E010B5074A002391809A
:1026F00053800A4601460548FDF71EFD044841681F
:1027000002221143416010BD64000020D00000206F
:102710000000054010B50021E12000F0EBF8002199
:10272000E22000F0E7F810BD10B57021272000F07E
:10273000E1F810BDFFB50D463EA003C887B001917A
:1027400000903EA000683EA1049003C9039102904E
:102750003DA0006805903DA0006806901E465A21E5
:10276000532000F0C7F8A521532000F0C3F801243E
:10277000374F02E03846FDF7ADFC641EFAD2FFF792
:10278000C9FFFFF7D1FF212E01D2002100E018215F
:102790003D2000F0AFF80021FD2000F0ABF8032150
:1027A000222000F0A7F8A81EC1B2232000F0A2F852
:1027B0002520099900F09EF83146312000F09AF862
:1027C0003146322000F096F82A463020079900F072
:1027D0007BF82A462A20079900F076F805226946F8
:1027E0003F2000F071F8062202A93A2000F06CF8B0
:1027F000012205A9392000F067F8032204A93E2030
:1028000000F062F8032206A93B2000F05DF80021E9
:102810003C2000F06FF82620109900F06BF80021A2
:10282000242000F067F80021212000F063F80BB0AD
:10283000F0BD000012ED679C46000000F63F5D0011
:102840004521EF2C5A400000010000000BDF020080
:102850000861000010B58F21202000F04BF8002106
:10286000FD2000F047F810BD70B50C46054600216C
:10287000FD2000F03FF84B200001FDF72BFC224625
:102880002946A02000F020F80748816A0029FCD1E1
:10289000FFF74AFF0021E12000F02CF80021FD2085
:1028A00000F028F870BD00008042005010B58E2165
:1028B000202000F01FF80021FD2000F01BF8F02080
:1028C000FDF708FC10BD0000F8B50F46084E0021CA
:1028D00015467160FFF784FD002404E0385DFFF7C2
:1028E0007FFD641CE4B2AC42F8D301207060F8BDF7
:1028F0000042005070B50D46054C00216160FFF7A5
:102900006FFD2846FFF76CFD0120606070BD000080
:102910000042005034290000000000207000000038
:102920008A100000A4290000700000209802000016
:102930009A10000000805101008051010000000049
:10294000000000000000000055CC5A00000000000C
:102950000000000000000000640090015802200305
:102960001212121212121212131212121312121245
:102970001212121212131212121312121212121235
:1029800012121312121213120000000000000000B5
:102990000000000000000000000000000000000037
:0429A0000000000033
:04000005000000F9FE
:00000001FF
